:10000000000000308A00412803178D0083168C13EE
:100010000C1483120C083C2803178C0083168C13D5
:100020000C1555308D00AA308D008C148C181628B4
:100030000C113C28A301A200FF30A207031CA30758
:10004000031C3C280330A100DF3028201C28A1011C
:10005000E83EA000A109FC30031C3128A0070318CA
:100060002E28A0070000A10F2E2820183728A01C3A
:100070003B2800003B280800831383120313000071
:10008000080083168501FF308600FF308700880155
:10009000831201308A010420A50002308A01042065
:1000A000A60003308A010420A70004308A0104203E
:1000B000A80005308A010420A90006308A01042026
:1000C000AA0007308A010420AB0008308A0104200E
:1000D000AC0009308A010420AD000A308A010420F6
:1000E000AE000B308A010420AF000C308A010420DE
:1000F000B0000D308A010420B1000E308A010420C6
:10010000B2000F308A010420B30010308A010420AD
:10011000B40011308A010420B50012308A01042095
:10012000B60013308A010420B70014308A0104207D
:10013000B80015308A010420B90016308A01042065
:10014000BA0017308A010420BB0018308A0104204D
:10015000BC0019308A010420BD001A308A01042035
:10016000BE001B308A010420BF001C308A0104201D
:10017000C0001D308A010420C1001E308A01042005
:10018000C2001F308A010420C30020308A010420ED
:10019000C40021308A010420C50022308A010420D5
:1001A000C60023308A010420C70024308A010420BD
:1001B000C80025308A010420C90026308A010420A5
:1001C000CA0027308A010420CB0028308A0104208D
:1001D000CC0029308A010420CD002A308A01042075
:1001E000CE002B308A010420CF002C308A0104205D
:1001F000D0002D308A010420D1002E308A01042045
:10020000D2002F308A010420D30030308A0104202C
:10021000D40031308A010420D50032308A01042014
:10022000D60033308A010420D70034308A010420FC
:10023000D80035308A010420D90036308A010420E4
:10024000DA0037308A010420DB0038308A010420CC
:10025000DC0039308A010420DD003A308A010420B4
:10026000DE003B308A010420DF003C308A0104209C
:10027000E0003D308A010420E1003E308A01042084
:10028000E2003F308A010420E30040308A0104206C
:10029000E40041308A010420E50042308A01042054
:1002A000E60043308A010420E70044308A0104203C
:1002B000E80045308A010420E90046308A01042024
:1002C000EA0047308A010420EB0048308A0104200C
:1002D000EC0049308A010420ED004A308A010420F4
:1002E000EE004B308A010420EF004C308A010420DC
:1002F000F0004D308A010420F1004E308A010420C4
:10030000F2004F308A010420F30050308A010420AB
:10031000F40051308A010420F50052308A01042093
:10032000F60053308A010420F70054308A0104207B
:10033000F80055308A010420F90056308A01042063
:10034000FA0057308A010420FB0058308A0104204B
:10035000FC0059308A010420FD005A308A01042033
:10036000FE005B308A010420FF005C308A0104201B
:100370008316A0005D3083128A0104208316A10039
:100380005E3083128A0104208316A2005F3083123C
:100390008A0104208316A300603083128A0104209E
:1003A0008316A400613083128A0104208316A500FD
:1003B000623083128A0104208316A6006330831200
:1003C0008A0104208316A700643083128A01042066
:1003D0008316A8007E3083128A0104208316AB00A6
:1003E000831203170D0A03138A0104208316AC003D
:1003F000803083128A0104208316A9000130AA00EC
:100400008A110A1283120618082A8A110A12AD2EBE
:100410008A110A1206190F2A8A110A16392985012A
:1004200025088A110A12031D182A8A110A12B82EE9
:10043000013083162A028A110A128312031D222A0E
:1004400025088800023083162A028A110A128312B4
:10045000031D2C2A26088800033083162A028A11DD
:100460000A128312031D362A2708880004308316D7
:100470002A028A110A128312031D402A28088800C2
:10048000053083162A028A110A128312031D4A2A92
:1004900029088800063083162A028A110A1283125C
:1004A000031D542A2A088800073083162A028A115D
:1004B0000A128312031D5E2A2B0888000830831657
:1004C0002A028A110A128312031D682A2C08880046
:1004D000093083162A028A110A128312031D722A16
:1004E0002D0888000A3083162A028A110A12831204
:1004F000031D7C2A2E0888000B3083162A028A11DD
:100500000A128312031D862A2F0888000C308316D6
:100510002A028A110A128312031D902A30088800C9
:100520000D3083162A028A110A128312031D9A2A99
:10053000310888000E3083162A028A110A128312AB
:10054000031DA42A320888000F3083162A028A115C
:100550000A128312031DAE2A330888001030831656
:100560002A028A110A128312031DB82A340888004D
:10057000113083162A028A110A128312031DC22A1D
:1005800035088800123083162A028A110A12831253
:10059000031DCC2A36088800133083162A028A11DC
:1005A0000A128312031DD62A3708880014308316D6
:1005B0002A028A110A128312031DE02A38088800D1
:1005C000153083162A028A110A128312031DEA2AA1
:1005D00039088800163083162A028A110A128312FB
:1005E000031DF42A3A088800173083162A028A115C
:1005F0000A128312031DFE2A3B0888001830831656
:100600002A028A110A128312031D082B3C08880053
:10061000193083162A028A110A128312031D122B23
:100620003D0888001A3083162A028A110A128312A2
:10063000031D1C2B3E0888001B3083162A028A11DA
:100640000A128312031D262B3F0888001C308316D4
:100650002A028A110A128312031D302B40088800D7
:100660001D3083162A028A110A128312031D3A2BA7
:10067000410888001E3083162A028A110A1283124A
:10068000031D442B420888001F3083162A028A115A
:100690000A128312031D4E2B430888002030831654
:1006A0002A028A110A128312031D582B440888005B
:1006B000213083162A028A110A128312031D622B2B
:1006C00045088800223083162A028A110A128312F2
:1006D000031D6C2B46088800233083162A028A11DA
:1006E0000A128312031D762B4708880024308316D4
:1006F0002A028A110A128312031D802B48088800DF
:10070000253083162A028A110A128312031D8A2BAE
:1007100049088800263083162A028A110A12831299
:10072000031D942B4A088800273083162A028A1159
:100730000A128312031D9E2B4B0888002830831653
:100740002A028A110A128312031DA82B4C08880062
:10075000293083162A028A110A128312031DB22B32
:100760004D0888002A3083162A028A110A12831241
:10077000031DBC2B4E0888002B3083162A028A11D9
:100780000A128312031DC62B4F0888002C308316D3
:100790002A028A110A128312031DD02B50088800E6
:1007A0002D3083162A028A110A128312031DDA2BB6
:1007B000510888002E3083162A028A110A128312E9
:1007C000031DE42B520888002F3083162A028A1159
:1007D0000A128312031DEE2B530888003030831653
:1007E0002A028A110A128312031DF82B540888006A
:1007F000313083162A028A110A128312031D022C39
:1008000055088800323083162A028A110A12831290
:10081000031D0C2C56088800333083162A028A11D7
:100820000A128312031D162C5708880034308316D1
:100830002A028A110A128312031D202C58088800EC
:10084000353083162A028A110A128312031D2A2CBC
:1008500059088800363083162A028A110A12831238
:10086000031D342C5A088800373083162A028A1157
:100870000A128312031D3E2C5B0888003830831651
:100880002A028A110A128312031D482C5C08880070
:10089000393083162A028A110A128312031D522C40
:1008A0005D0888003A3083162A028A110A128312E0
:1008B000031D5C2C5E0888003B3083162A028A11D7
:1008C0000A128312031D662C5F0888003C308316D1
:1008D0002A028A110A128312031D702C60088800F4
:1008E0003D3083162A028A110A128312031D7A2CC4
:1008F000610888003E3083162A028A110A12831288
:10090000031D842C620888003F3083162A028A1156
:100910000A128312031D8E2C630888004030831650
:100920002A028A110A128312031D982C6408880077
:10093000413083162A028A110A128312031DA22C47
:1009400065088800423083162A028A110A1283122F
:10095000031DAC2C66088800433083162A028A11D6
:100960000A128312031DB62C6708880044308316D0
:100970002A028A110A128312031DC02C68088800FB
:10098000453083162A028A110A128312031DCA2CCB
:1009900069088800463083162A028A110A128312D7
:1009A000031DD42C6A088800473083162A028A1156
:1009B0000A128312031DDE2C6B0888004830831650
:1009C0002A028A110A128312031DE82C6C0888007F
:1009D000493083162A028A110A128312031DF22C4F
:1009E0006D0888004A3083162A028A110A1283127F
:1009F000031DFC2C6E0888004B3083162A028A11D6
:100A00000A128312031D062D6F0888004C308316CE
:100A10002A028A110A128312031D102D7008880001
:100A20004D3083162A028A110A128312031D1A2DD1
:100A3000710888004E3083162A028A110A12831226
:100A4000031D242D720888004F3083162A028A1154
:100A50000A128312031D2E2D73088800503083164E
:100A60002A028A110A128312031D382D7408880085
:100A7000513083162A028A110A128312031D422D55
:100A800075088800523083162A028A110A128312CE
:100A9000031D4C2D76088800533083162A028A11D4
:100AA0000A128312031D562D7708880054308316CE
:100AB0002A028A110A128312031D602D7808880009
:100AC000553083162A028A110A128312031D6A2DD9
:100AD00079088800563083162A028A110A12831276
:100AE000031D742D7A088800573083162A028A1154
:100AF0000A128312031D7E2D7B088800583083164E
:100B00002A028A110A128312031D882D7C0888008C
:100B1000593083162A028A110A128312031D922D5C
:100B20007D0888005A3083162A028A110A1283121D
:100B3000031D9C2D7E0888005B3083162A028A11D3
:100B40000A128312031DA62D7F0888005C308316CD
:100B50002A028A110A128312031DB22D831620085D
:100B6000831288005D3083162A028A110A128312CA
:100B7000031DBE2D83162108831288005E30831664
:100B80002A028A110A128312031DCA2D8316220813
:100B9000831288005F3083162A028A110A12831298
:100BA000031DD62D83162308831288006030831618
:100BB0002A028A110A128312031DE22D83162408C9
:100BC00083128800613083162A028A110A12831266
:100BD000031DEE2D831625088312880062308316CC
:100BE0002A028A110A128312031DFA2D831626087F
:100BF00083128800633083162A028A110A12831234
:100C0000031D062E8316270883128800643083167E
:100C10002A028A110A128312031D122E8316280833
:100C20008312880083162C088312A30083162B08D6
:100C300083128A011B208A110A120618222E8A1199
:100C40000A12AD2E8316AA0A2A0829028A110A124C
:100C50008312031D2E2E01308316AA0083128A11DF
:100C60000A128619382E64308316AB070318AC0AB3
:100C700083128A110A12061A442E32308316AB02EE
:100C80000030031C013EAC02831283162C088A112B
:100C90000A128312031D582E323083162B028A113A
:100CA0000A1283120318582E8316AC013230AB009F
:100CB0008312073083162C028A110A128312031C36
:100CC000722E8A110A12031D6D2ED13083162B024B
:100CD0008A110A128312031C722E07308316AC008D
:100CE000D030AB0083128A110A1286187A2E8A1528
:100CF0000A1643258A110A120619812E8A150A1628
:100D00005E258A110A128619962E7E3003178D00F1
:100D1000831603132B0883128A010C2003178D0AF4
:100D2000831603132C0883128A010C208A110A12DD
:100D3000061AAB2E7E3003178D00831603132B0883
:100D400083128A010C2003178D0A831603132C08C3
:100D500083128A010C208A010F2A01308500C830D5
:100D60008A011A208A110A120618B82E8A01AD2E9D
:100D7000013085008A110A128619C12E8A110A16BD
:100D8000262C8A110A120718C92E013088068316EC
:100D9000081083128A110A128718D22E0230880690
:100DA0008316881083128A110A120719DB2E043069
:100DB00088068316081183128A110A128719E42EF5
:100DC000083088068316881183128A110A12071ABE
:100DD000ED2E103088068316081283128A110A122B
:100DE000871AF62E203088068316881283128A11FD
:100DF0000A12071BFF2E4030880683160813831241
:100E00008A110A12871B082F8030880683168813E0
:100E10008312C8308A011A20013083162A028A11EF
:100E20000A128312031D162F0808A500023083162C
:100E30002A028A110A128312031D202F0808A60015
:100E4000033083162A028A110A128312031D2A2FE5
:100E50000808A700043083162A028A110A12831296
:100E6000031D342F0808A800053083162A028A11B2
:100E70000A128312031D3E2F0808A90006308316AC
:100E80002A028A110A128312031D482F0808AA0099
:100E9000073083162A028A110A128312031D522F69
:100EA0000808AB00083083162A028A110A1283123E
:100EB000031D5C2F0808AC00093083162A028A1132
:100EC0000A128312031D662F0808AD000A3083162C
:100ED0002A028A110A128312031D702F0808AE001D
:100EE0000B3083162A028A110A128312031D7A2FED
:100EF0000808AF000C3083162A028A110A128312E6
:100F0000031D842F0808B0000D3083162A028A11B1
:100F10000A128312031D8E2F0808B1000E308316AB
:100F20002A028A110A128312031D982F0808B200A0
:100F30000F3083162A028A110A128312031DA22F70
:100F40000808B300103083162A028A110A1283128D
:100F5000031DAC2F0808B400113083162A028A1131
:100F60000A128312031DB62F0808B500123083162B
:100F70002A028A110A128312031DC02F0808B60024
:100F8000133083162A028A110A128312031DCA2FF4
:100F90000808B700143083162A028A110A12831235
:100FA000031DD42F0808B800153083162A028A11B1
:100FB0000A128312031DDE2F0808B90016308316AB
:100FC0002A028A110A128312031DE82F0808BA00A8
:100FD000173083162A028A110A128312031DF22F78
:100FE0000808BB00183083162A028A110A128312DD
:100FF000031DFC2F0808BC00193083162A028A152D
:101000000A128312031D06280808BD001A30831631
:101010002A028A150A128312031D10280808BE002E
:101020001B3083162A028A150A128312031D1A28FE
:101030000808BF001C3083162A028A150A12831280
:10104000031D24280808C0001D3083162A028A15B3
:101050000A128312031D2E280808C1001E308316B1
:101060002A028A150A128312031D38280808C200B2
:101070001F3083162A028A150A128312031D422882
:101080000808C300203083162A028A150A12831228
:10109000031D4C280808C400213083162A028A1533
:1010A0000A128312031D56280808C5002230831631
:1010B0002A028A150A128312031D60280808C60036
:1010C000233083162A028A150A128312031D6A2806
:1010D0000808C700243083162A028A150A128312D0
:1010E000031D74280808C800253083162A028A15B3
:1010F0000A128312031D7E280808C90026308316B1
:101100002A028A150A128312031D88280808CA00B9
:10111000273083162A028A150A128312031D922889
:101120000808CB00283083162A028A150A12831277
:10113000031D9C280808CC00293083162A028A1532
:101140000A128312031DA6280808CD002A30831630
:101150002A028A150A128312031DB0280808CE003D
:101160002B3083162A028A150A128312031DBA280D
:101170000808CF002C3083162A028A150A1283121F
:10118000031DC4280808D0002D3083162A028A15B2
:101190000A128312031DCE280808D1002E308316B0
:1011A0002A028A150A128312031DD8280808D200C1
:1011B0002F3083162A028A150A128312031DE22891
:1011C0000808D300303083162A028A150A128312C7
:1011D000031DEC280808D400313083162A028A1532
:1011E0000A128312031DF6280808D5003230831630
:1011F0002A028A150A128312031D00290808D60044
:10120000333083162A028A150A128312031D0A2913
:101210000808D700343083162A028A150A1283126E
:10122000031D14290808D800353083162A028A15B0
:101230000A128312031D1E290808D90036308316AE
:101240002A028A150A128312031D28290808DA00C7
:10125000373083162A028A150A128312031D322997
:101260000808DB00383083162A028A150A12831216
:10127000031D3C290808DC00393083162A028A1530
:101280000A128312031D46290808DD003A3083162E
:101290002A028A150A128312031D50290808DE004B
:1012A0003B3083162A028A150A128312031D5A291B
:1012B0000808DF003C3083162A028A150A128312BE
:1012C000031D64290808E0003D3083162A028A15B0
:1012D0000A128312031D6E290808E1003E308316AE
:1012E0002A028A150A128312031D78290808E200CF
:1012F0003F3083162A028A150A128312031D82299F
:101300000808E300403083162A028A150A12831265
:10131000031D8C290808E400413083162A028A152F
:101320000A128312031D96290808E500423083162D
:101330002A028A150A128312031DA0290808E60052
:10134000433083162A028A150A128312031DAA2922
:101350000808E700443083162A028A150A1283120D
:10136000031DB4290808E800453083162A028A15AF
:101370000A128312031DBE290808E90046308316AD
:101380002A028A150A128312031DC8290808EA00D6
:10139000473083162A028A150A128312031DD229A6
:1013A0000808EB00483083162A028A150A128312B5
:1013B000031DDC290808EC00493083162A028A152F
:1013C0000A128312031DE6290808ED004A3083162D
:1013D0002A028A150A128312031DF0290808EE005A
:1013E0004B3083162A028A150A128312031DFA292A
:1013F0000808EF004C3083162A028A150A1283125D
:10140000031D042A0808F0004D3083162A028A15AD
:101410000A128312031D0E2A0808F1004E308316AB
:101420002A028A150A128312031D182A0808F200DC
:101430004F3083162A028A150A128312031D222AAC
:101440000808F300503083162A028A150A12831204
:10145000031D2C2A0808F400513083162A028A152D
:101460000A128312031D362A0808F500523083162B
:101470002A028A150A128312031D402A0808F60060
:10148000533083162A028A150A128312031D4A2A30
:101490000808F700543083162A028A150A128312AC
:1014A000031D542A0808F800553083162A028A15AD
:1014B0000A128312031D5E2A0808F90056308316AB
:1014C0002A028A150A128312031D682A0808FA00E4
:1014D000573083162A028A150A128312031D722AB4
:1014E0000808FB00583083162A028A150A12831254
:1014F000031D7C2A0808FC00593083162A028A152D
:101500000A128312031D862A0808FD005A3083162A
:101510002A028A150A128312031D902A0808FE0067
:101520005B3083162A028A150A128312031D9A2A37
:101530000808FF005C3083162A028A150A128312FB
:10154000031DA52A08088316A00083125D308316A8
:101550002A028A150A128312031DB12A080883166B
:10156000A10083125E3083162A028A150A128312A2
:10157000031DBD2A08088316A20083125F3083165C
:101580002A028A150A128312031DC92A0808831623
:10159000A3008312603083162A028A150A1283126E
:1015A000031DD52A08088316A40083126130831610
:1015B0002A028A150A128312031DE12A08088316DB
:1015C000A5008312623083162A028A150A1283123A
:1015D000031DED2A08088316A600831263308316C4
:1015E0002A028A150A128312031DF92A0808831693
:1015F000A7008312643083162A028A150A12831206
:10160000031D052B08088316A80083128A150A12E9
:1016100006180D2B8A150A12242B8A150A12861811
:10162000142B8A150A123E238A150A1206191B2B3F
:101630008A110A1639298A150A12061A222B8A11CA
:101640000A16542C8A01B82E8501C8308A011A2046
:101650008A150A1206182F2B8A150A12242B8316B4
:101660002A0AA9008030831203178D008316031302
:10167000290883128A010C208A014828023085003B
:10168000C8308A011A208A150A1286184A2B8A1530
:101690000A123E2B013083162A028A150A1283127F
:1016A000031D592B013003178D00031325088A01F0
:1016B0000C20023083162A028A150A128312031D97
:1016C000682B023003178D00031326088A010C20B3
:1016D000033083162A028A150A128312031D772B00
:1016E000033003178D00031327088A010C200430F0
:1016F00083162A028A150A128312031D862B0430D0
:1017000003178D00031328088A010C200530831667
:101710002A028A150A128312031D952B053003171E
:101720008D00031329088A010C20063083162A0233
:101730008A150A128312031DA42B063003178D008D
:1017400003132A088A010C20073083162A028A15FF
:101750000A128312031DB32B073003178D000313E6
:101760002B088A010C20083083162A028A150A12D7
:101770008312031DC22B083003178D0003132C089E
:101780008A010C20093083162A028A150A12831254
:10179000031DD12B093003178D0003132D088A0177
:1017A0000C200A3083162A028A150A128312031D9E
:1017B000E02B0A3003178D0003132E088A010C203A
:1017C0000B3083162A028A150A128312031DEF2B8F
:1017D0000B3003178D0003132F088A010C200C30E7
:1017E00083162A028A150A128312031DFE2B0C305F
:1017F00003178D00031330088A010C200D30831667
:101800002A028A150A128312031D0D2C0D300317AC
:101810008D00031331088A010C200E3083162A0232
:101820008A150A128312031D1C2C0E3003178D001B
:10183000031332088A010C200F3083162A028A15FE
:101840000A128312031D2B2C0F3003178D00031374
:1018500033088A010C20103083162A028A150A12D6
:101860008312031D3A2C103003178D000313340824
:101870008A010C20113083162A028A150A1283125B
:10188000031D492C113003178D00031335088A01FD
:101890000C20123083162A028A150A128312031DA5
:1018A000582C123003178D00031336088A010C20C0
:1018B000133083162A028A150A128312031D672C1D
:1018C000133003178D00031337088A010C201430DE
:1018D00083162A028A150A128312031D762C1430ED
:1018E00003178D00031338088A010C201530831666
:1018F0002A028A150A128312031D852C153003173C
:101900008D00031339088A010C20163083162A0231
:101910008A150A128312031D942C163003178D00AA
:1019200003133A088A010C20173083162A028A15FD
:101930000A128312031DA32C173003178D00031303
:101940003B088A010C20183083162A028A150A12D5
:101950008312031DB22C183003178D0003133C08AB
:101960008A010C20193083162A028A150A12831262
:10197000031DC12C193003178D0003133D088A0184
:101980000C201A3083162A028A150A128312031DAC
:10199000D02C1A3003178D0003133E088A010C2047
:1019A0001B3083162A028A150A128312031DDF2CAC
:1019B0001B3003178D0003133F088A010C201C30D5
:1019C00083162A028A150A128312031DEE2C1C307C
:1019D00003178D00031340088A010C201D30831665
:1019E0002A028A150A128312031DFD2C1D300317CB
:1019F0008D00031341088A010C201E3083162A0231
:101A00008A150A128312031D0C2D1E3003178D0038
:101A1000031342088A010C201F3083162A028A15FC
:101A20000A128312031D1B2D1F3003178D00031391
:101A300043088A010C20203083162A028A150A12D4
:101A40008312031D2A2D203003178D000313440831
:101A50008A010C20213083162A028A150A12831269
:101A6000031D392D213003178D00031345088A010A
:101A70000C20223083162A028A150A128312031DB3
:101A8000482D223003178D00031346088A010C20CD
:101A9000233083162A028A150A128312031D572D3A
:101AA000233003178D00031347088A010C202430CC
:101AB00083162A028A150A128312031D662D24300A
:101AC00003178D00031348088A010C202530831664
:101AD0002A028A150A128312031D752D2530031759
:101AE0008D00031349088A010C20263083162A0230
:101AF0008A150A128312031D842D263003178D00C8
:101B000003134A088A010C20273083162A028A15FB
:101B10000A128312031D932D273003178D00031320
:101B20004B088A010C20283083162A028A150A12D3
:101B30008312031DA22D283003178D0003134C08B8
:101B40008A010C20293083162A028A150A12831270
:101B5000031DB12D293003178D0003134D088A0191
:101B60000C202A3083162A028A150A128312031DBA
:101B7000C02D2A3003178D0003134E088A010C2054
:101B80002B3083162A028A150A128312031DCF2DC9
:101B90002B3003178D0003134F088A010C202C30C3
:101BA00083162A028A150A128312031DDE2D2C3099
:101BB00003178D00031350088A010C202D30831663
:101BC0002A028A150A128312031DED2D2D300317E8
:101BD0008D00031351088A010C202E3083162A022F
:101BE0008A150A128312031DFC2D2E3003178D0057
:101BF000031352088A010C202F3083162A028A15FB
:101C00000A128312031D0B2E2F3003178D000313AE
:101C100053088A010C20303083162A028A150A12D2
:101C20008312031D1A2E303003178D00031354083E
:101C30008A010C20313083162A028A150A12831277
:101C4000031D292E313003178D00031355088A0117
:101C50000C20323083162A028A150A128312031DC1
:101C6000382E323003178D00031356088A010C20DA
:101C7000333083162A028A150A128312031D472E57
:101C8000333003178D00031357088A010C203430BA
:101C900083162A028A150A128312031D562E343027
:101CA00003178D00031358088A010C203530831662
:101CB0002A028A150A128312031D652E3530031776
:101CC0008D00031359088A010C20363083162A022E
:101CD0008A150A128312031D742E363003178D00E5
:101CE00003135A088A010C20373083162A028A15FA
:101CF0000A128312031D832E373003178D0003133E
:101D00005B088A010C20383083162A028A150A12D1
:101D10008312031D922E383003178D0003135C08C5
:101D20008A010C20393083162A028A150A1283127E
:101D3000031DA12E393003178D0003135D088A019E
:101D40000C203A3083162A028A150A128312031DC8
:101D5000B02E3A3003178D0003135E088A010C2061
:101D60003B3083162A028A150A128312031DBF2EE6
:101D70003B3003178D0003135F088A010C203C30B1
:101D800083162A028A150A128312031DCE2E3C30B6
:101D900003178D00031360088A010C203D30831661
:101DA0002A028A150A128312031DDD2E3D30031705
:101DB0008D00031361088A010C203E3083162A022D
:101DC0008A150A128312031DEC2E3E3003178D0074
:101DD000031362088A010C203F3083162A028A15F9
:101DE0000A128312031DFB2E3F3003178D000313CD
:101DF00063088A010C20403083162A028A150A12D1
:101E00008312031D0A2F403003178D00031364084B
:101E10008A010C20413083162A028A150A12831285
:101E2000031D192F413003178D00031365088A0124
:101E30000C20423083162A028A150A128312031DCF
:101E4000282F423003178D00031366088A010C20E7
:101E5000433083162A028A150A128312031D372F74
:101E6000433003178D00031367088A010C204430A8
:101E700083162A028A150A128312031D462F443044
:101E800003178D00031368088A010C204530831660
:101E90002A028A150A128312031D552F4530031793
:101EA0008D00031369088A010C20463083162A022C
:101EB0008A150A128312031D642F463003178D0002
:101EC00003136A088A010C20473083162A028A15F8
:101ED0000A128312031D732F473003178D0003135B
:101EE0006B088A010C20483083162A028A150A12D0
:101EF0008312031D822F483003178D0003136C08D3
:101F00008A010C20493083162A028A150A1283128C
:101F1000031D912F493003178D0003136D088A01AB
:101F20000C204A3083162A028A150A128312031DD6
:101F3000A02F4A3003178D0003136E088A010C206E
:101F40004B3083162A028A150A128312031DAF2F03
:101F50004B3003178D0003136F088A010C204C309F
:101F600083162A028A150A128312031DBE2F4C30D3
:101F700003178D00031370088A010C204D3083165F
:101F80002A028A150A128312031DCD2F4D30031722
:101F90008D00031371088A010C204E3083162A022B
:101FA0008A150A128312031DDC2F4E3003178D0091
:101FB000031372088A010C204F3083162A028A15F7
:101FC0000A128312031DEB2F4F3003178D000313EA
:101FD00073088A010C20503083162A028A150A12CF
:101FE0008312031DFA2F503003178D00031374085A
:101FF0008A010C20513083162A028A110A16831294
:10200000031D0928513003178D00031375088A0139
:102010000C20523083162A028A110A168312031DDD
:102020001828523003178D00031376088A010C20FC
:10203000533083162A028A110A168312031D272899
:10204000533003178D00031377088A010C20543096
:1020500083162A028A110A168312031D3628543069
:1020600003178D00031378088A010C20553083165E
:102070002A028A110A168312031D452855300317B8
:102080008D00031379088A010C20563083162A022A
:102090008A110A168312031D5428563003178D0027
:1020A00003137A088A010C20573083162A028A11FA
:1020B0000A168312031D6328573003178D0003137C
:1020C0007B088A010C20583083162A028A110A16CE
:1020D0008312031D7228583003178D0003137C08E8
:1020E0008A010C20593083162A028A110A1683129B
:1020F000031D8128593003178D0003137D088A01C1
:102100000C205A3083162A028A110A168312031DE4
:1021100090285A3003178D0003137E088A010C2083
:102120005B3083162A028A110A168312031D9F2828
:102130005B3003178D0003137F088A010C205C308D
:1021400083162A028A110A168312031DB0285C30F6
:1021500003178D0083160313200883128A010C20B5
:102160005D3083162A028A110A168312031DC128C4
:102170005D3003178D0083160313210883128A0133
:102180000C205E3083162A028A110A168312031D60
:10219000D2285E3003178D008316031322088312A2
:1021A0008A010C205F3083162A028A110A168312D4
:1021B000031DE3285F3003178D00831603132308E4
:1021C00083128A010C20603083162A028A110A16B3
:1021D0008312031DF428603003178D008316031348
:1021E000240883128A010C20613083162A028A1186
:1021F0000A168312031D0529613003178D0083160B
:102200000313250883128A010C20623083162A02E8
:102210008A110A168312031D1629623003178D00D6
:1022200083160313260883128A010C206330831659
:102230002A028A110A168312031D27296330031705
:102240008D0083160313270883128A010C20643043
:1022500083162A028A110A168312031D3829643054
:1022600003178D0083160313280883128A010C209C
:10227000080004308500C8308A011A208A110A1625
:10228000061945298A110A163929013003178D00CC
:10229000030103138A010C20023003178D00030190
:1022A00003138A010C20033003178D00030103136D
:1022B0008A010C20043003178D00030103138A01E7
:1022C0000C20053003178D00030103138A010C2035
:1022D000063003178D00030103138A010C20073019
:1022E00003178D00030103138A010C200830031724
:1022F0008D00030103138A010C20093003178D00A0
:10230000030103138A010C200A3003178D00030117
:1023100003138A010C200B3003178D0003010313F4
:102320008A010C200C3003178D00030103138A016E
:102330000C200D3003178D00030103138A010C20BC
:102340000E3003178D00030103138A010C200F3098
:1023500003178D00030103138A010C2010300317AB
:102360008D00030103138A010C20113003178D0027
:10237000030103138A010C20123003178D0003019F
:1023800003138A010C20133003178D00030103137C
:102390008A010C20143003178D00030103138A01F6
:1023A0000C20153003178D00030103138A010C2044
:1023B000163003178D00030103138A010C20173018
:1023C00003178D00030103138A010C201830031733
:1023D0008D00030103138A010C20193003178D00AF
:1023E000030103138A010C201A3003178D00030127
:1023F00003138A010C201B3003178D000301031304
:102400008A010C201C3003178D00030103138A017D
:102410000C201D3003178D00030103138A010C20CB
:102420001E3003178D00030103138A010C201F3097
:1024300003178D00030103138A010C2020300317BA
:102440008D00030103138A010C20213003178D0036
:10245000030103138A010C20223003178D000301AE
:1024600003138A010C20233003178D00030103138B
:102470008A010C20243003178D00030103138A0105
:102480000C20253003178D00030103138A010C2053
:10249000263003178D00030103138A010C20273017
:1024A00003178D00030103138A010C202830031742
:1024B0008D00030103138A010C20293003178D00BE
:1024C000030103138A010C202A3003178D00030136
:1024D00003138A010C202B3003178D000301031313
:1024E0008A010C202C3003178D00030103138A018D
:1024F0000C202D3003178D00030103138A010C20DB
:102500002E3003178D00030103138A010C202F3096
:1025100003178D00030103138A010C2030300317C9
:102520008D00030103138A010C20313003178D0045
:10253000030103138A010C20323003178D000301BD
:1025400003138A010C20333003178D00030103139A
:102550008A010C20343003178D00030103138A0114
:102560000C20353003178D00030103138A010C2062
:10257000363003178D00030103138A010C20373016
:1025800003178D00030103138A010C203830031751
:102590008D00030103138A010C20393003178D00CD
:1025A000030103138A010C203A3003178D00030145
:1025B00003138A010C203B3003178D000301031322
:1025C0008A010C203C3003178D00030103138A019C
:1025D0000C203D3003178D00030103138A010C20EA
:1025E0003E3003178D00030103138A010C203F3096
:1025F00003178D00030103138A010C2040300317D9
:102600008D00030103138A010C20413003178D0054
:10261000030103138A010C20423003178D000301CC
:1026200003138A010C20433003178D0003010313A9
:102630008A010C20443003178D00030103138A0123
:102640000C20453003178D00030103138A010C2071
:10265000463003178D00030103138A010C20473015
:1026600003178D00030103138A010C204830031760
:102670008D00030103138A010C20493003178D00DC
:10268000030103138A010C204A3003178D00030154
:1026900003138A010C204B3003178D000301031331
:1026A0008A010C204C3003178D00030103138A01AB
:1026B0000C204D3003178D00030103138A010C20F9
:1026C0004E3003178D00030103138A010C204F3095
:1026D00003178D00030103138A010C2050300317E8
:1026E0008D00030103138A010C20513003178D0064
:1026F000030103138A010C20523003178D000301DC
:1027000003138A010C20533003178D0003010313B8
:102710008A010C20543003178D00030103138A0132
:102720000C20553003178D00030103138A010C2080
:10273000563003178D00030103138A010C20573014
:1027400003178D00030103138A010C20583003176F
:102750008D00030103138A010C20593003178D00EB
:10276000030103138A010C205A3003178D00030163
:1027700003138A010C205B3003178D000301031340
:102780008A010C205C3003178D00030103138A01BA
:102790000C205D3003178D00030103138A010C2008
:1027A0005E3003178D00030103138A010C205F3094
:1027B00003178D00030103138A010C2060300317F7
:1027C0008D00030103138A010C20613003178D0073
:1027D000030103138A010C20623003178D000301EB
:1027E00003138A010C20633003178D0003010313C8
:1027F0008A010C20643003178D00030103138A0142
:102800000C20803003178D00643003138A010C20E4
:1028100003308316AC002030AB007E3083120317E8
:102820008D00831603132B0883128A010C200317D3
:102830008D0A831603132C0883128A010C200130A1
:102840008316AA0083128A110A16852CC8308A01C1
:102850001A208A110A168619302C8A110A16262C7B
:102860008316AA032A088A110A168312031D3A2C1A
:102870000730850083162A088A110A168312031D61
:10288000462C0330A300E8308A011B2083162A0857
:102890008A110A168312031D502C01308316AA00D8
:1028A00083128A110A16852CC8308A011A208A11CF
:1028B0000A16061A5E2C8A110A16542C8316AA0AC6
:1028C00065302A028A110A168312031C692C07300C
:1028D0008500653083162A028A110A168312031CAA
:1028E000762C0330A300E8308A011B206530831664
:1028F0002A028A110A168312031C812C6430831663
:10290000AA0083128A110A16852C013083162A0226
:102910008A110A168312031D912C01308A010420AA
:10292000A500023083162A028A110A168312031D9B
:102930009D2C02308A010420A600033083162A024F
:102940008A110A168312031DA92C03308A01042060
:10295000A700043083162A028A110A168312031D67
:10296000B52C04308A010420A800053083162A0201
:102970008A110A168312031DC12C05308A01042016
:10298000A900063083162A028A110A168312031D33
:10299000CD2C06308A010420AA00073083162A02B3
:1029A0008A110A168312031DD92C07308A010420CC
:1029B000AB00083083162A028A110A168312031DFF
:1029C000E52C08308A010420AC00093083162A0265
:1029D0008A110A168312031DF12C09308A01042082
:1029E000AD000A3083162A028A110A168312031DCB
:1029F000FD2C0A308A010420AE000B3083162A0217
:102A00008A110A168312031D092D0B308A01042036
:102A1000AF000C3083162A028A110A168312031D96
:102A2000152D0C308A010420B0000D3083162A02C7
:102A30008A110A168312031D212D0D308A010420EC
:102A4000B1000E3083162A028A110A168312031D62
:102A50002D2D0E308A010420B2000F3083162A0279
:102A60008A110A168312031D392D0F308A010420A2
:102A7000B300103083162A028A110A168312031D2E
:102A8000452D10308A010420B400113083162A022B
:102A90008A110A168312031D512D11308A01042058
:102AA000B500123083162A028A110A168312031DFA
:102AB0005D2D12308A010420B600133083162A02DD
:102AC0008A110A168312031D692D13308A0104200E
:102AD000B700143083162A028A110A168312031DC6
:102AE000752D14308A010420B800153083162A028F
:102AF0008A110A168312031D812D15308A010420C4
:102B0000B900163083162A028A110A168312031D91
:102B10008D2D16308A010420BA00173083162A0240
:102B20008A110A168312031D992D17308A01042079
:102B3000BB00183083162A028A110A168312031D5D
:102B4000A52D18308A010420BC00193083162A02F2
:102B50008A110A168312031DB12D19308A0104202F
:102B6000BD001A3083162A028A110A168312031D29
:102B7000BD2D1A308A010420BE001B3083162A02A4
:102B80008A110A168312031DC92D1B308A010420E5
:102B9000BF001C3083162A028A110A168312031DF5
:102BA000D52D1C308A010420C0001D3083162A0256
:102BB0008A110A168312031DE12D1D308A0104209B
:102BC000C1001E3083162A028A110A168312031DC1
:102BD000ED2D1E308A010420C2001F3083162A0208
:102BE0008A110A168312031DF92D1F308A01042051
:102BF000C300203083162A028A110A168312031D8D
:102C0000052E20308A010420C400213083162A02B8
:102C10008A110A168312031D112E21308A01042005
:102C2000C500223083162A028A110A168312031D58
:102C30001D2E22308A010420C600233083162A026A
:102C40008A110A168312031D292E23308A010420BB
:102C5000C700243083162A028A110A168312031D24
:102C6000352E24308A010420C800253083162A021C
:102C70008A110A168312031D412E25308A01042071
:102C8000C900263083162A028A110A168312031DF0
:102C90004D2E26308A010420CA00273083162A02CE
:102CA0008A110A168312031D592E27308A01042027
:102CB000CB00283083162A028A110A168312031DBC
:102CC000652E28308A010420CC00293083162A0280
:102CD0008A110A168312031D712E29308A010420DD
:102CE000CD002A3083162A028A110A168312031D88
:102CF0007D2E2A308A010420CE002B3083162A0232
:102D00008A110A168312031D892E2B308A01042092
:102D1000CF002C3083162A028A110A168312031D53
:102D2000952E2C308A010420D0002D3083162A02E3
:102D30008A110A168312031DA12E2D308A01042048
:102D4000D1002E3083162A028A110A168312031D1F
:102D5000AD2E2E308A010420D2002F3083162A0295
:102D60008A110A168312031DB92E2F308A010420FE
:102D7000D300303083162A028A110A168312031DEB
:102D8000C52E30308A010420D400313083162A0247
:102D90008A110A168312031DD12E31308A010420B4
:102DA000D500323083162A028A110A168312031DB7
:102DB000DD2E32308A010420D600333083162A02F9
:102DC0008A110A168312031DE92E33308A0104206A
:102DD000D700343083162A028A110A168312031D83
:102DE000F52E34308A010420D800353083162A02AB
:102DF0008A110A168312031D012F35308A0104201F
:102E0000D900363083162A028A110A168312031D4E
:102E10000D2F36308A010420DA00373083162A025B
:102E20008A110A168312031D192F37308A010420D4
:102E3000DB00383083162A028A110A168312031D1A
:102E4000252F38308A010420DC00393083162A020D
:102E50008A110A168312031D312F39308A0104208A
:102E6000DD003A3083162A028A110A168312031DE6
:102E70003D2F3A308A010420DE003B3083162A02BF
:102E80008A110A168312031D492F3B308A01042040
:102E9000DF003C3083162A028A110A168312031DB2
:102EA000552F3C308A010420E0003D3083162A0271
:102EB0008A110A168312031D612F3D308A010420F6
:102EC000E1003E3083162A028A110A168312031D7E
:102ED0006D2F3E308A010420E2003F3083162A0223
:102EE0008A110A168312031D792F3F308A010420AC
:102EF000E300403083162A028A110A168312031D4A
:102F0000852F40308A010420E400413083162A02D4
:102F10008A110A168312031D912F41308A01042061
:102F2000E500423083162A028A110A168312031D15
:102F30009D2F42308A010420E600433083162A0286
:102F40008A110A168312031DA92F43308A01042017
:102F5000E700443083162A028A110A168312031DE1
:102F6000B52F44308A010420E800453083162A0238
:102F70008A110A168312031DC12F45308A010420CD
:102F8000E900463083162A028A110A168312031DAD
:102F9000CD2F46308A010420EA00473083162A02EA
:102FA0008A110A168312031DD92F47308A01042083
:102FB000EB00483083162A028A110A168312031D79
:102FC000E52F48308A010420EC00493083162A029C
:102FD0008A110A168312031DF12F49308A01042039
:102FE000ED004A3083162A028A110A168312031D45
:102FF000FD2F4A308A010420EE004B3083162A024E
:103000008A150A168312031D09284B308A010420F1
:10301000EF004C3083162A028A150A168312031D0C
:1030200015284C308A010420F0004D3083162A0206
:103030008A150A168312031D21284D308A010420A7
:10304000F1004E3083162A028A150A168312031DD8
:103050002D284E308A010420F2004F3083162A02B8
:103060008A150A168312031D39284F308A0104205D
:10307000F300503083162A028A150A168312031DA4
:10308000452850308A010420F400513083162A026A
:103090008A150A168312031D512851308A01042013
:1030A000F500523083162A028A150A168312031D70
:1030B0005D2852308A010420F600533083162A021C
:1030C0008A150A168312031D692853308A010420C9
:1030D000F700543083162A028A150A168312031D3C
:1030E000752854308A010420F800553083162A02CE
:1030F0008A150A168312031D812855308A0104207F
:10310000F900563083162A028A150A168312031D07
:103110008D2856308A010420FA00573083162A027F
:103120008A150A168312031D992857308A01042034
:10313000FB00583083162A028A150A168312031DD3
:10314000A52858308A010420FC00593083162A0231
:103150008A150A168312031DB12859308A010420EA
:10316000FD005A3083162A028A150A168312031D9F
:10317000BD285A308A010420FE005B3083162A02E3
:103180008A150A168312031DC9285B308A010420A0
:10319000FF005C3083162A028A150A168312031D6B
:1031A000D6285C308A0104208316A00083125D308B
:1031B00083162A028A150A168312031DE4285D303D
:1031C0008A0104208316A10083125E3083162A022E
:1031D0008A150A168312031DF2285E308A01042024
:1031E0008316A20083125F3083162A028A150A16FC
:1031F0008312031D00295F308A0104208316A30077
:103200008312603083162A028A150A168312031D60
:103210000E2960308A0104208316A40083126130D5
:1032200083162A028A150A168312031D1C2961308F
:103230008A0104208316A5008312623083162A02B5
:103240008A150A168312031D2A2962308A01042076
:103250008316A6008312633083162A028A150A1683
:103260008312031D382963308A0104208316A700C6
:103270008312643083162A028A150A168312031DEC
:10328000462964308A0104208316A8008312013085
:1032900083162A028A150A168312031D512925084E
:1032A0008800023083162A028A150A168312031D2B
:1032B0005B2926088800033083162A028A150A161D
:1032C0008312031D652927088800043083162A020B
:1032D0008A150A168312031D6F29280888000530F5
:1032E00083162A028A150A168312031D79292908D2
:1032F0008800063083162A028A150A168312031DD7
:1033000083292A088800073083162A028A150A169C
:103310008312031D8D292B088800083083162A028A
:103320008A150A168312031D97292C088800093074
:1033300083162A028A150A168312031DA1292D0855
:1033400088000A3083162A028A150A168312031D82
:10335000AB292E0888000B3083162A028A150A161C
:103360008312031DB5292F0888000C3083162A020A
:103370008A150A168312031DBF29300888000D30F4
:1033800083162A028A150A168312031DC9293108D9
:1033900088000E3083162A028A150A168312031D2E
:1033A000D329320888000F3083162A028A150A169C
:1033B0008312031DDD2933088800103083162A028A
:1033C0008A150A168312031DE72934088800113074
:1033D00083162A028A150A168312031DF12935085D
:1033E0008800123083162A028A150A168312031DDA
:1033F000FB2936088800133083162A028A150A161C
:103400008312031D052A37088800143083162A0208
:103410008A150A168312031D0F2A380888001530F2
:1034200083162A028A150A168312031D192A3908DF
:103430008800163083162A028A150A168312031D85
:10344000232A3A088800173083162A028A150A169A
:103450008312031D2D2A3B088800183083162A0288
:103460008A150A168312031D372A3C088800193072
:1034700083162A028A150A168312031D412A3D0863
:1034800088001A3083162A028A150A168312031D31
:103490004B2A3E0888001B3083162A028A150A161A
:1034A0008312031D552A3F0888001C3083162A0208
:1034B0008A150A168312031D5F2A400888001D30F2
:1034C00083162A028A150A168312031D692A4108E7
:1034D00088001E3083162A028A150A168312031DDD
:1034E000732A420888001F3083162A028A150A169A
:1034F0008312031D7D2A43088800203083162A0288
:103500008A150A168312031D872A44088800213071
:1035100083162A028A150A168312031D912A45086A
:103520008800223083162A028A150A168312031D88
:103530009B2A46088800233083162A028A150A1619
:103540008312031DA52A47088800243083162A0207
:103550008A150A168312031DAF2A480888002530F1
:1035600083162A028A150A168312031DB92A4908EE
:103570008800263083162A028A150A168312031D34
:10358000C32A4A088800273083162A028A150A1699
:103590008312031DCD2A4B088800283083162A0287
:1035A0008A150A168312031DD72A4C088800293071
:1035B00083162A028A150A168312031DE12A4D0872
:1035C00088002A3083162A028A150A168312031DE0
:1035D000EB2A4E0888002B3083162A028A150A1619
:1035E0008312031DF52A4F0888002C3083162A0207
:1035F0008A150A168312031DFF2A500888002D30F1
:1036000083162A028A150A168312031D092B5108F4
:1036100088002E3083162A028A150A168312031D8B
:10362000132B520888002F3083162A028A150A1697
:103630008312031D1D2B53088800303083162A0285
:103640008A150A168312031D272B5408880031306F
:1036500083162A028A150A168312031D312B550878
:103660008800323083162A028A150A168312031D37
:103670003B2B56088800333083162A028A150A1617
:103680008312031D452B57088800343083162A0205
:103690008A150A168312031D4F2B580888003530EF
:1036A00083162A028A150A168312031D592B5908FC
:1036B0008800363083162A028A150A168312031DE3
:1036C000632B5A088800373083162A028A150A1697
:1036D0008312031D6D2B5B088800383083162A0285
:1036E0008A150A168312031D772B5C08880039306F
:1036F00083162A028A150A168312031D812B5D0880
:1037000088003A3083162A028A150A168312031D8E
:103710008B2B5E0888003B3083162A028A150A1616
:103720008312031D952B5F0888003C3083162A0204
:103730008A150A168312031D9F2B600888003D30EE
:1037400083162A028A150A168312031DA92B610803
:1037500088003E3083162A028A150A168312031D3A
:10376000B32B620888003F3083162A028A150A1696
:103770008312031DBD2B63088800403083162A0284
:103780008A150A168312031DC72B6408880041306E
:1037900083162A028A150A168312031DD12B650887
:1037A0008800423083162A028A150A168312031DE6
:1037B000DB2B66088800433083162A028A150A1616
:1037C0008312031DE52B67088800443083162A0204
:1037D0008A150A168312031DEF2B680888004530EE
:1037E00083162A028A150A168312031DF92B69080B
:1037F0008800463083162A028A150A168312031D92
:10380000032C6A088800473083162A028A150A1694
:103810008312031D0D2C6B088800483083162A0282
:103820008A150A168312031D172C6C08880049306C
:1038300083162A028A150A168312031D212C6D088D
:1038400088004A3083162A028A150A168312031D3D
:103850002B2C6E0888004B3083162A028A150A1614
:103860008312031D352C6F0888004C3083162A0202
:103870008A150A168312031D3F2C700888004D30EC
:1038800083162A028A150A168312031D492C710811
:1038900088004E3083162A028A150A168312031DE9
:1038A000532C720888004F3083162A028A150A1694
:1038B0008312031D5D2C73088800503083162A0282
:1038C0008A150A168312031D672C7408880051306C
:1038D00083162A028A150A168312031D712C750895
:1038E0008800523083162A028A150A168312031D95
:1038F0007B2C76088800533083162A028A150A1614
:103900008312031D852C77088800543083162A0201
:103910008A150A168312031D8F2C780888005530EB
:1039200083162A028A150A168312031D992C790818
:103930008800563083162A028A150A168312031D40
:10394000A32C7A088800573083162A028A150A1693
:103950008312031DAD2C7B088800583083162A0281
:103960008A150A168312031DB72C7C08880059306B
:1039700083162A028A150A168312031DC12C7D089C
:1039800088005A3083162A028A150A168312031DEC
:10399000CB2C7E0888005B3083162A028A150A1613
:1039A0008312031DD52C7F0888005C3083162A0201
:1039B0008A150A168312031DE12C83162008831230
:1039C00088005D3083162A028A150A168312031DA9
:1039D000ED2C83162108831288005E3083162A029C
:1039E0008A150A168312031DF92C831622088312E6
:1039F00088005F3083162A028A150A168312031D77
:103A0000052D8316230883128800603083162A024E
:103A10008A150A168312031D112D8316240883129A
:103A20008800613083162A028A150A168312031D44
:103A30001D2D8316250883128800623083162A0202
:103A40008A150A168312031D292D83162608831250
:103A50008800633083162A028A150A168312031D12
:103A6000352D8316270883128800643083162A02B6
:103A70008A150A168312031D412D83162808831206
:103A800088008A01B82E03308316AC002030AB00CA
:103A90007E30831203178D00831603132B088312C5
:103AA0008A010C2003178D0A831603132C08831236
:103AB0008A010C20C8308A011A20080001308316C0
:103AC000AA00C83083128A011A208A150A1606191C
:0A3AD0006C2D8A150A165E2D080001
:02400E003A3F37
:00000001FF
